:1000000000308A007D280000FF00030E8301A3005A
:100010007F08A2000A08A7008A01A20E0408A40013
:100020002008A5002108A600831383128C308400C9
:10003000801E1C288C1A2928240884002508A0006A
:100040002608A10027088A00230E8300FF0E7F0EDA
:1000500009008A112B282830480784008C1E2E287E
:10006000140880004808CD00013048071F39C80037
:1000700049084802031D3E284D08C8008C128A1109
:100080001C284908480203194128283049078400E0
:100090000008CA00013049071F39C9004A08A100F9
:1000A0008A11A72883168711831287110830A100AF
:1000B000000000000000A1176C28A113CC0C03184D
:1000C0008715031C871121176C282113A10B5E28AB
:1000D00000000000000087150E308400840B6E289D
:1000E00000000000A11B5D28211B65288A117B28C8
:1000F0004B08CC0052288A11A22884011F308305A6
:100100001F1300308316910007308312990071305D
:1001100083168F000F0887118312871591110C30F9
:1001200093002230960090309700C801C9011F1338
:1001300000308316910083121F1083168C16C03076
:1001400083128B04490848020319AB28412821086F
:0A015000CA00CB007828A228630043
:02400E00C43FAD
:00000001FF
